:020000040800F2
:10000000000200203D08000879290008492900085D
:1000100065290008492900085D2900083F080008F3
:100020003F0800083F0800083F0800087139000831
:100030003F0800083F0800083F0800087545000811
:100040003F0800083F0800083F0800083F08000874
:100050003F0800083F080008A9420008D5420008F0
:10006000014300082D430008594300083F080008D9
:100070003F0800083F0800083F0800083F08000844
:100080003F0800083F0800083F080008FD28000856
:1000900029290008392900083F080008854300087D
:1000A0003F0800083F0800083F0800083F08000814
:1000B0003F0800083F0800083F0800083F08000804
:1000C0003F0800083F0800083F0800083F080008F4
:1000D0003F0800083F0800083F0800083F080008E4
:1000E000ED4300083F0800083F0800083F080008EB
:1000F0003F0800083F0800083F0800083F080008C4
:100100003F0800083F0800083F0800083F080008B3
:100110003F0800083F0800083F0800083F080008A3
:100120003F0800083F0800083F0800083F08000893
:100130003F0800083F0800083F0800083F08000883
:100140003F0800083F0800083F0800083F08000873
:100150003F0800083F0800083F0800083F08000863
:10016000AD150008000000000000000000000000C5
:100170004FF0FF0C1CEAD0521EBF1CEAD15392EA8A
:100180000C0F93EA0C0F6FD01A4480EA010C400266
:1001900018BF5FEA41211ED04FF0006343EA5010C0
:1001A00043EA5111A0FB01310CF00040B1F5000F02
:1001B0003EBF490041EAD3715B0040EA010062F1B1
:1001C0007F02FD2A1DD8B3F1004F40EBC25008BF9B
:1001D00020F00100704790F0000F0CF0004C08BFB9
:1001E00049024CEA502040EA51207F3AC2BFD2F186
:1001F000FF0340EAC250704740F400004FF0000394
:10020000013A5DDC12F1190FDCBF00F000407047CD
:10021000C2F10002410021FA02F1C2F1200200FA0B
:1002200002FC5FEA310040F1000053EA4C0308BFD2
:1002300020EADC70704792F0000F00F0004C02BF23
:10024000400010F4000F013AF9D040EA0C0093F09E
:10025000000F01F0004C02BF490011F4000F013BF8
:10026000F9D041EA0C018FE70CEAD15392EA0C0F66
:1002700018BF93EA0C0F0AD030F0004C18BF31F0D1
:10028000004CD8D180EA010000F00040704790F0A7
:10029000000F17BF90F0004F084691F0000F91F04B
:1002A000004F14D092EA0C0F01D142020FD193EA11
:1002B0000C0F03D14B0218BF084608D180EA010099
:1002C00000F0004040F0FE4040F40000704740F075
:1002D000FE4040F44000704780F0004002E000BF64
:1002E00081F0004142001FBF5FEA410392EA030F21
:1002F0007FEA226C7FEA236C6AD04FEA1262D2EB6B
:100300001363C1BFD218414048404140B8BF5B426F
:10031000192B88BF704710F0004F40F4000020F008
:100320007F4018BF404211F0004F41F4000121F01E
:100330007F4118BF494292EA030F3FD0A2F1010268
:1003400041FA03FC10EB0C00C3F1200301FA03F1A6
:1003500000F0004302D5494260EB4000B0F5000FC9
:1003600013D3B0F1807F06D340084FEA310102F188
:100370000102FE2A51D2B1F1004F40EBC25008BF3A
:1003800020F0010040EA03007047490040EB000004
:10039000013A28BFB0F5000FEDD2B0FA80FCACF105
:1003A000080CB2EB0C0200FA0CF0AABF00EBC25032
:1003B00052421843BCBFD0401843704792F0000F20
:1003C00081F4000106BF80F400000132013BB5E773
:1003D0004FEA41037FEA226C18BF7FEA236C21D0E9
:1003E00092EA030F04D092F0000F08BF084670474E
:1003F00090EA010F1CBF0020704712F07F4F04D11C
:10040000400028BF40F00040704712F100723CBF2E
:1004100000F50000704700F0004343F0FE4040F458
:10042000000070477FEA226216BF08467FEA236316
:100430000146420206BF5FEA412390EA010F40F401
:10044000800070474FF0000304E000BF10F000434D
:1004500048BF40425FEA000C08BF704743F0964334
:1004600001464FF000001CE050EA010208BF70474F
:100470004FF000030AE000BF50EA010208BF7047D6
:1004800011F0004302D5404261EB41015FEA010CEB
:1004900002BF84460146002043F0B64308BFA3F1E3
:1004A0008053A3F50003BCFA8CF2083AA3EBC253C5
:1004B00010DB01FA02FC634400FA02FCC2F12002E4
:1004C000BCF1004F20FA02F243EB020008BF20F01B
:1004D0000100704702F1200201FA02FCC2F1200281
:1004E00050EA4C0021FA02F243EB020008BF20EA76
:1004F000DC70704742000ED2B2F1FE4F0BD34FF0CA
:100500009E03B3EB126209D44FEA002343F0004389
:1005100023FA02F070474FF00000704712F1610FAC
:1005200001D1420202D14FF0FF3070474FF000007E
:10053000704700BF53B94AB9002908BF00281CBF43
:100540004FF0FF314FF0FF3000F076B9ADF1080CFD
:100550006DE904CE00F006F8DDF804E0DDE90223E1
:1005600004B070472DE9F047089E0D4604468846C2
:10057000002B4DD18A42944668D9B2FA82F252B128
:1005800001FA02F3C2F1200120FA01F10CFA02FC97
:1005900041EA030894404FEA1C41B8FBF1F71FFA07
:1005A0008CFE01FB178807FB0EF0230C43EA08437F
:1005B00098420AD91CEB030307F1FF3580F01E8136
:1005C000984240F21B81023F63441B1AB3FBF1F0D7
:1005D00001FB103300FB0EFEA4B244EA0344A6451F
:1005E0000AD91CEB040400F1FF3380F00981A64511
:1005F00040F20681644402380021A4EB0E0440EA74
:1006000007401EB10023D440C6E90043BDE8F0878F
:100610008B4208D9002E00F0EE800021C6E90005CB
:100620000846BDE8F087B3FA83F100294AD1AB420E
:1006300002D3824200F2FC80841A65EB030301209E
:100640009846002EE2D0C6E90048DFE702B9FFDE97
:10065000B2FA82F2002A40F09180A1EB0C00012155
:100660004FEA1C471FFA8CFEB0FBF7F307FB1300A1
:10067000250C45EA00450EFB03F0A84208D91CEB07
:10068000050503F1FF3802D2A84200F2CE804346AE
:100690002D1AB5FBF7F007FB10550EFB00FEA4B2B8
:1006A00044EA0544A64508D91CEB040400F1FF35D3
:1006B00002D2A64500F2B6802846A4EB0E0440EA1A
:1006C00003409EE7C1F120078B4022FA07FC4CEA69
:1006D000030C25FA07FA4FEA1C49BAFBF9F820FA8D
:1006E00007F309FB18AA8D401FFA8CFE1D4300FA80
:1006F00001F308FB0EF02C0C44EA0A44A04202FA73
:1007000001F20BD91CEB040408F1FF3A80F0888059
:10071000A04240F28580A8F102086444241AB4FB88
:10072000F9F009FB104400FB0EFEADB245EA0444AB
:10073000A64508D91CEB040400F1FF356CD2A64590
:100740006AD90238644440EA0840A0FB0295A4EB51
:100750000E04AC42C846AE4656D353D0002E69D0E4
:10076000B3EB080264EB0E0422FA01F304FA07F774
:100770001F43CC40C6E90074002147E70CFA02FC95
:10078000C2F1200125FA01F34FEA1C4720FA01F1DA
:1007900095400D43B3FBF7F107FB11331FFA8CFEB5
:1007A000280C40EA034001FB0EF3834204FA02F4F2
:1007B00008D91CEB000001F1FF382FD283422DD95C
:1007C00002396044C01AB0FBF7F307FB1300ADB267
:1007D00045EA004503FB0EF0A84208D91CEB0505CD
:1007E00003F1FF3816D2A84214D9023B6544281AF7
:1007F00043EA014138E73146304607E72F46E4E651
:100800001846F9E64B45A9D2B9EB020865EB0C0E88
:100810000138A3E74346EAE7284694E74146D1E793
:10082000D0467BE76444023847E7023B65442FE744
:10083000084606E73146E9E6704700BF02E000F0EF
:1008400000F8FEE772B6264880F30888254880F352
:100850000988254825490860022080F31488BFF3E1
:100860006F8F03F045FC03F0A9FC4FF05530204991
:100870001B4A91423CBF41F8040BFAE71D49194A53
:1008800091423CBF41F8040BFAE71B491B4A1C4B41
:100890009A423EBF51F8040B42F8040BF8E70020DF
:1008A0001849194A91423CBF41F8040BFAE703F09A
:1008B00023FC03F085FC154C154DAC4203DA54F8CB
:1008C000041B8847F9E700F03FF8124C124DAC4288
:1008D00003DA54F8041B8847F9E703F00BBC000067
:1008E00000020020000800200000000808ED00E0E1
:1008F000000100200002002010480008000800202D
:1009000080080020800800203025002060010008B9
:100910006401000864010008640100082DE9F04F3B
:10092000C1F80CD0C3689D46BDE8F08F002383F367
:1009300011882846A047002003F096F9FEE703F04F
:10094000F9F800DFFEE70000F8B500F041FE314A9B
:10095000536823F0E06343F0905343F480435360C3
:1009600003F060FB074603F0AFFB0546C8BB2A4B0C
:100970009F4236D001339F4236D0284B27F0FF02EA
:100980009A4234D1F8B200F03BFC2E4642F2107489
:1009900000F03CFC08B10024264601F00FF950B3EA
:1009A0000024032000F03EF8264635B11C4B9F4240
:1009B00003D0002403F080FB2646002003F03CFB1C
:1009C0000EB100F045F800F08DFC00F003FE01F0E0
:1009D000DBFF0546ACB900F0CDFC012003F04AF97D
:1009E000F8E72E460024D3E704460126D0E7064662
:1009F00041F28834CCE7002CD7D04FF47A7401262A
:100A0000D3E701F0C1FF431BA342E4D900F020F873
:100A1000DDE700BF00000140010007B0000008B0A2
:100A2000263A09B0084B187003280CD8DFE800F00C
:100A300008050208022000F035BE022000F02ABEA0
:100A40000022024B5A607047800800208408002072
:100A500038B501F0B3F830B103221F4B1A700022F1
:100A60001E4B5A6038BD1E4B1E4A19680131F9D021
:100A700004339342F9D11C4C194DD4F80428AA42EE
:100A8000F0D31A4B9B6803F1006303F508439A42C5
:100A9000E8D203F0E5FA03F0F7FA002000F0C0FD19
:100AA0000220FFF7BFFF124BDA690022DA61D96931
:100AB00099699A619B6972B64FF0E023C3F8085DAB
:100AC0003021D4F80038D4F8042881F311889D46E9
:100AD00083F308881047C5E78008002084080020B9
:100AE0000088000820880008008000080008002016
:100AF0000010024049F26900084A136899B21B0CC1
:100B000000FB013344F250611360054B186882B258
:100B1000000C01FB0200186080B27047180800202A
:100B20001408002010B504460021102200F0D6FD64
:100B3000034B03CB206061601868A06010BD00BF4C
:100B4000E8F7FF1F2DE9F0410026ADF54E7D6CACB6
:100B500040F2751207460D460EA831460D9600F07C
:100B6000BDFD4FF4C4723146204600F0B7FD01F0E0
:100B70000BFF4FF47A72B0FBF2F0264B0DF1340804
:100B8000186093E80700022384E807000DF5E97078
:100B90002382FFF7C7FF4EF603531F4907A823849C
:100BA00003F0B4FD17230DF2E32284F832310DF186
:100BB0002C0C07AB1E4603CE6645106051603346D1
:100BC00002F10802F6D130681060B188B37920468E
:100BD000918093714146012200F0CCFD00230393E4
:100BE000AB7E80B2029305F1190301930123CDE995
:100BF00004800093384605A3D3E90023E97E02F080
:100C000087FA0DF54E7DBDE8F08100BF9E6AC421D4
:100C1000818A46EE8C0800201C4700082DE9F0412F
:100C20002C4C8046237A0D46DAB05BBB284627A9B8
:100C300000F0B0FE0746002842D19DF89D60C82E06
:100C40003ED801464FF4A662204600F047FD4FF41F
:100C50008073C4F8F8314FF40073C4F80C334FF4C8
:100C600040733246C4F820340DF19E0104F10900AE
:100C700000F022FD9DF89C302644777223720BB958
:100C8000EB7E23728122002106AC27A800F026FD0E
:100C90000122214627A800F0B9FE00230393AB7E72
:100CA00080B2029305F1190301932823CDE9044092
:100CB0000093404605A3D3E90023E97E02F028FA19
:100CC0005AB0BDE8F08100BFAFF3008026417272D8
:100CD000DF25D7B7A81D0020F0B54FF48A75002492
:100CE000234EF1B005FB006596F8D830D822214696
:100CF00085F8DC3085F8E8403AA800F0EFFC06F112
:100D0000090000F0E3FCD5F8E430C2B206AF8DF87C
:100D1000F00006F109010DF1F100CDE93A3400F0DF
:100D2000CBFC394601223AA800F09CFE80B2CDE906
:100D3000047008230127CDE9023706F1D803019397
:100D40003023317A00930B4807A3D3E9002302F044
:100D5000DFF9A04206DD01F017FEC5F8E0003846D5
:100D600071B0F0BD2046FBE778F6339F93CACD8D76
:100D7000A81D0020A41800202DE9F0411D4D1E4E95
:100D80001E4F86B0284602F0EFF9034658B3002400
:100D9000CDE90344ADF81440027B02948DF8142091
:100DA0009968406803AA03C21B68DFF8548043F0C7
:100DB0000043029301F0EAFD821941F10003384635
:100DC000009402A901F0D6F8A04205DD284602F001
:100DD000CFF988F80040D5E798F80030072B05D800
:100DE000013388F8003006B0BDE8F081014802F018
:100DF000BFF9F8E7A418002040420F00D8180020DF
:100E0000DD22002070B50D4614461E4602F0DCF8C7
:100E100050B9022E10D1012C0ED112A3D3E9002318
:100E20000120C5E9002307E0282C10D005D8012CAB
:100E300009D0052C0FD0002070BD302CFBD10BA3A6
:100E4000D3E90023ECE70BA3D3E90023E8E70BA3E6
:100E5000D3E90023E4E70BA3D3E90023E0E700BFD5
:100E6000AFF30080401DA12026812A0B78F6339F26
:100E700093CACD8D9E6AC421818A46EE2641727244
:100E8000DF25D7B7F017304A39059E5638B50546E5
:100E90000E4C0021013500F0E5FBA4F82C55B4F808
:100EA0002C0500F0C7FB78B1B4F82C0500F0D2FB9C
:100EB000014648B9B4F82C0500F0D4FBB4F82C3541
:100EC0000133A4F82C35EAE738BD00BFA81D002087
:100ED00010B50A4B0A4A1A6093F8602442B9D3F855
:100EE0005C442CB1204600F0E7FE204603F050FBA6
:100EF000BDE81040034800F0DFBE00BFD818002056
:100F000070470008201D00202DE9F04F8FB000AF82
:100F100005460C4602F058F8002848D1237E022BE3
:100F20001AD1E38A012B17D101F02EFD0646FFF7F7
:100F3000E1FD4FF4C873B0FBF3F202FB1303DFF8DB
:100F4000A0829BB206F516763344C8F80030E37EE3
:100F500033B90022A34B1A703C37BD46BDE8F08F71
:100F6000204607F1240100F0D3FC0028F4D107F15A
:100F70001400FFF7D7FD97F8264007F11401224629
:100F800007F1270003F04EFB0028E2D10F2C08D810
:100F9000944B1C70D8F80030A3F51673C8F80030D5
:100FA000DAE7284697F8241002F006F8D4E7E38A37
:100FB000282B2BD010D8012B23D0052BCCD1BFF35D
:100FC0004F8F8949894BCA6802F4E0621343CB60B2
:100FD000BFF34F8F00BFFDE7302BBDD1844EE17EC4
:100FE000327A9142B8D131460022607E91F8DC50CD
:100FF000854200F0A5800132042A01F58A71F5D1FD
:10100000AAE721462846FFF79DFDA5E72146284689
:10101000FFF704FEA0E7B2F8EC507B6005F103098E
:101020004FEA99094FEA8902D11DC908A8EBC1030B
:101030009D46EB460021584600F050FB04F1EE01BE
:101040002A465846314400F037FB7B6813B901202B
:1010500000F0E6FA96F8D20000F0ECFA044630B957
:10106000307200F007FB204600F0DAFAB0E0D6F864
:10107000D4203AB996F8D200B6F82C25824201D88D
:10108000FFF704FFD6F8D4202A44944208D296F8F9
:10109000D200B6F82C250130824201D8FFF7F6FEC7
:1010A000594670685FFA89F200F020FB08B9C5461E
:1010B00078E0726896F8D2002A447260D6F8D4209C
:1010C00005EB0209C6F8D49000F0B4FA814509D3C3
:1010D00096F8D220D6F8D4000132001B86F8D22030
:1010E000C6F8D400FF2D0FD80024347200F0C2FAE5
:1010F000204600F095FA00F061FD3E4B188108B9DA
:10110000FFF7A6FCC54627E7BB6896F8D9000AFB9F
:101110000362D2F8E410FB6801F5806182F8E830E0
:10112000C2F8E030C2F8E410FFF7D6FDFFF724FE66
:1011300096F8D920013202F0030286F8D920B6E7EA
:101140004FF48A7A0AFB02F505F1EA0120463144A0
:1011500000F0B4FCF86000287FF4FEAE01223544B4
:1011600085F8E82001F010FCD5F8E020801A192855
:1011700040F6B83238BF1920904228BF1046FFF71A
:1011800061F91D49FEF7F4FF04463068FFF75AF98C
:101190001A49FEF7EDFF01462046FFF7A3F8FFF7D7
:1011A000A9F9306096F8D930BB60BA6873680AFB59
:1011B00002F4321992F8E81059B1D2F8E410E84676
:1011C0008B423FF428AF002182F8E810C2F8E0100B
:1011D000C5467368074A9B0A01331381BCE600BF0A
:1011E000A01800209D18002000ED00E00400FA0582
:1011F000A81D00208C080020CDCCCC3D6666663F43
:10120000014B1870704700BF9808002030B54FF0B0
:1012100000542B4B226885B09A4207D002F05EFF43
:10122000044620BB0024204605B030BD627D254B1E
:1012300025481A70237D002503724FF48073C0F88F
:10124000F8314FF40073C0F80C334FF44073C922E7
:10125000C0F820341D49C0F8E450093000F02CFAE1
:101260002046E022294600F039FA0124DBE7184A3B
:10127000184DD36943F00073D361AA6D164B9A429F
:10128000D0D12B6E013B7E2BCCD8144A01AB07CAC0
:1012900083E807001846032100F060FC6B6D834271
:1012A0004FF00003BED12A6D8A4203BFAB652A6EA0
:1012B000044B1C4601BF1A70EA6D094B1A60B2E775
:1012C0009AAD44C598080020A81D002016000020F3
:1012D00000100240006600405041A0B05866004037
:1012E0001008002037B500F069FC0223184D0122D8
:1012F0006B71184B28811968174801F0F3F9002326
:101300000193164B164900934FF48052154B164823
:1013100001F028FE154B197811B1134801F04CFE6D
:1013200001F032FB0446FFF7E5FB4FF4C873B0FB56
:10133000F3F202FB130304F516709BB218440C4B36
:10134000186002F0C1FE08B10F232B8103B030BD3D
:101350008C08002010080020D8180020050E000876
:101360009C080020090F0008A418002098080020FD
:10137000A01800202DE9F04F0FF22829D9E90089A3
:101380007E4C93B0FFF7F8FC00230BAE7C4FDFF8E8
:10139000F4A10A93ADF834300B9373604FF0000B57
:1013A000002200230125CDE9002338465B460DF1DC
:1013B0001D0207A98DF81C508DF81DB001F044F9ED
:1013C0009DF81C30002B40F0A080204601F0FCFD71
:1013D0000646002845D101F0D7FA6B4F3B6898428A
:1013E0003FD301F0D1FA8246FFF784FB4FF4C87374
:1013F000B0FBF3F202FB130083B20AF51670184437
:101400003860624F0EA897F800B0BBF1000F14BF10
:1014100033462B46CBF1100A5FFA8AFA8DF8283052
:10142000FFF780FBBAF1060F28BF4FF0060A0EAB9C
:1014300003EB0B0152460DF1290000F03DF90AAB18
:10144000039318230AF101020293514BD2B2CDE962
:1014500000530492204647A3D3E9002301F0FAFD8C
:101460003E7001F091FA4B4A4B4D1368C31AB3F525
:101470007A7F2ED3106001F089FA02460B4620468F
:1014800001F080FE204601F09FFD10B32B7A434E01
:10149000002B14BF03230223737101F075FA4FF47C
:1014A0007A73B0FBF3F00EAF01223060394630465C
:1014B00000F006FA18230293394B80B2019340F2F0
:1014C0005513CDE90370009342464B46204601F088
:1014D000C1FD2B7AB3B101F057FA002607464FF44D
:1014E0008A7A95F8D900304400F003000AFB0053D3
:1014F00093F8E8206AB30136042EF2D12B7A002B40
:101500007FF440AF13B0BDE8F08FDAF80C305946E5
:1015100083F00803CAF80C3010220EA800F0DEF8A1
:101520000DF11E0308AA0AA9384600F019FE96E834
:1015300003000FAB83E803009DF8343020468DF89C
:1015400044300A9B0EA90E93DDE9082301F0F0FF59
:1015500024E7D3F8E02042B12B68BA1AFA2B38BF3F
:10156000FA230533B2EB430FC5D3FFF7B5FB0028D1
:10157000C1D1C3E7401DA12026812A0BA418002059
:10158000D8180020000C0140A01800209D18002051
:101590009C180020D8220020A81D00208C080020C4
:1015A000DC220020F1C6A7C1D068080F08B50548A5
:1015B00000F06CFEBDE808400020034A034902F039
:1015C000E1BF00BFD818002018230020D10E00086A
:1015D0007047000070B502F0F9FB00250E4C0F4E6D
:1015E00020803068238883420CD800252088013869
:1015F00002F0E8FB23880544013BB5F5805F2380BA
:10160000F4D370BD02F0DEFB336805440133B5F559
:10161000084F3360E5D3E8E70C230020E0220020E8
:1016200002F062BC00F10060920000F5084002F098
:1016300007BC0000054B1A68054B1B889B1A8342A8
:1016400002D9104402F0BEBB00207047E022002007
:101650000C230020024B1B68184402F0B9BB00BFEA
:10166000E0220020024B1B68184402F0C3BB00BFFD
:10167000E0220020064991F8243033B100230822EB
:10168000086A81F82430FFF7CDBF0120704700BF02
:10169000E4220020022802BF0822014B1A61704791
:1016A000000C0140022802BF4FF40022014B1A61D6
:1016B000704700BF000C0140002310B5934203D0D7
:1016C000CC5CC4540133F9E710BD00000346024668
:1016D000D01A12F9011B0029FAD1704703460244BF
:1016E000934202D003F8011BFAE770472DE9F84353
:1016F0001F4D144695F824200746884652BBDFF854
:1017000070909CB395F824302BB92022FF214846D5
:101710002F62FFF7E3FF95F824004146C0F108026D
:10172000A24228BF224605EB8000D6B29200FFF706
:10173000C3FF95F82430A41B1E44F6B2082E1744AC
:101740009044E4B285F82460DBD1FFF793FF0028D2
:10175000D7D108E02B6A03EB82038342CFD0FFF797
:1017600089FF0028CBD10020BDE8F8830120FBE7EA
:10177000E42200202DE9F0470D4604460021904662
:10178000284640F27912FFF7A9FF234620220021C4
:10179000284601F06FFE022220212846231D01F079
:1017A00069FE032222212846631D01F063FE032205
:1017B00025212846A31D01F05DFE10222821284680
:1017C00004F1080301F056FE08223821284604F1EE
:1017D000100301F04FFE08224021284604F11103B6
:1017E00001F048FE08224821284604F1120301F0C6
:1017F00041FE20225021284604F1140301F03AFE54
:1018000040227021284604F1180301F033FE08221B
:10181000B021284604F1200301F02CFE0822B82153
:10182000284604F1210301F025FEC02604F1220719
:101830003B46314608222846083601F01BFEB6F525
:10184000A07F07F10107F3D108223146284604F1B1
:10185000320301F00FFE002704F1330A94F832300E
:101860004FEAC7099F4209F5A47615D3B8F1000FD6
:1018700008D131460722284604F5997301F0FAFD94
:1018800009F24F16274694F832213B1B93420CD3A2
:10189000F01DC008BDE8F0870AEB070308223146B7
:1018A000284601F0E7FD0137D8E7314607F2331348
:1018B0000822284601F0DEFD08360137E3E7000084
:1018C00038B50C460021054621600346C4F80310D4
:1018D0002046202201F0CEFD20462B1D0222202191
:1018E00001F0C8FD20466B1D0322222101F0C2FD3C
:1018F0002046AB1D0322252101F0BCFD204610220D
:10190000282105F1080301F0B5FD072038BD0000CE
:101910000023F7B50E460546047F072200911946BD
:1019200001F06AFC731C0093012200230721284662
:1019300001F062FCC4B9B31C0093052223460821C0
:10194000284601F059FC0D243746B278BB1B934260
:1019500011D32B7FE01DC008AC8ABBB9A04294BF55
:101960000020012003B0F0BDAB8A0824DB00083B57
:10197000DB08B370E8E7FB1C214600930822002334
:10198000284601F039FC08340137DEE7001B18BF98
:101990000120E7E70023F7B50E46047F08220091F7
:1019A0001946054601F028FC731CC4B908220093AF
:1019B00011462346284601F01FFC102401237278AB
:1019C0005F1C013B934211D32B7FE01DC008AC8A02
:1019D000BBB9A04294BF0020012003B0F0BDAB8A88
:1019E0000824DB00083BDB087370E7E7F3192146A6
:1019F000009308220023284601F0FEFB08343B46F2
:101A0000DDE7001B18BF0120E7E70000F8B50E4630
:101A100005461446002181223046FFF75FFE2B4623
:101A200008220021304601F025FD7CB9072208215B
:101A300030466B1C01F01EFD0F2401236A785F1CE9
:101A4000013B934204D3E01DC008F8BD0824F4E72D
:101A50002146EB190822304601F00CFD08343B46C4
:101A6000ECE70000F8B50E46054614460021CE22EC
:101A70003046FFF733FE2B4628220021304601F086
:101A8000F9FC7CB908222821304605F1080301F051
:101A9000F1FC30242F462A7A7B1B934204D3E01DAD
:101AA000C008F8BD2824F5E7214607F109030822FC
:101AB000304601F0DFFC08340137ECE7F7B5047F6E
:101AC0000E460091012310220021054601F094FBEF
:101AD000C4B9B31C0093092223461021284601F003
:101AE0008BFB192437467288BB1B9A4211D82B7F77
:101AF000E01DC008AC8ABBB9A04294BF0020012001
:101B000003B0F0BDAB8A1024DB00103BDB08738010
:101B1000E8E73B1D2146009308220023284601F0F8
:101B20006BFB08340137DEE7001B18BF0120E7E735
:101B300030B5094D0A4491420DD011F8013B58408F
:101B4000082340F30004013B2C4013F0FF0384EA18
:101B50005000F6D1EFE730BD2083B8ED4FF0FF33F2
:101B6000F7B500EB81061946DFF848C0DFF848E01A
:101B7000B0421BD050F8042B01AF0192042217F899
:101B8000014B81EA046108240D46DB184941013C00
:101B9000002DBCBF83EA0C0381EA0E0114F0FF04A0
:101BA000F2D1013A12F0FF02E9D1E1E7D843C9438B
:101BB00003B0F0BD9336EAA9EBE1F042F7B56B460E
:101BC000374A106851686A4603C3082335493648C6
:101BD00002F038FD0446002833D10A256B46334A0B
:101BE000106851686A4603C3082331492E4802F041
:101BF00029FD0446002849D00369B3F55E3F45D866
:101C000040F2ED32B0F8661091423FD1294A0244C9
:101C100002F15C018B4239D35C3B234900209E1AC0
:101C2000FFF786FF07463246002004F16401FFF704
:101C30007FFFA3689F4229D1E368984208BF00252F
:101C400024E00369B3F55E3F27D840F2ED32418BC3
:101C5000914220D1174A024402F110018B4218D35D
:101C6000103B114900209D1AFFF762FF06462A46E5
:101C7000002004F11801FFF75BFFA3689E4202D128
:101C8000E368984201D00D25A8E70025284603B057
:101C9000F0BD1025A2E70C25A0E70B259EE700BFAD
:101CA00034470008DC770300008800083D4700083F
:101CB000907703000878FFF710B5037C044613B94A
:101CC000006802F0A7FC204610BD00000023BFF30F
:101CD0005B8FC360BFF35B8FBFF35B8F8360BFF32A
:101CE0005B8F7047BFF35B8F0068BFF35B8F7047FC
:101CF00070B505460C30FFF7F5FF05F10806044600
:101D00003046FFF7EFFFA04206D930466D68FFF777
:101D1000E9FF2C44201A70BD3046FFF7E3FFF9E7D6
:101D200070B505464068A0B105F10800FFF7DAFF7D
:101D300005F10C0604463046FFF7D4FF844288BF05
:101D40000025304698BF6D68FFF7CCFF013C2C445E
:101D5000201A70BD38B50C460546FFF7C9FFA042F2
:101D600010D305F10800FFF7BDFF04446868BFF316
:101D70005B8FB4FBF0F100FB1144AC60BFF35B8FF1
:101D8000012038BD0020FCE72DE9F041144607464C
:101D90000D46FFF7C5FF844228BF0446D4B1B846BC
:101DA00058F80C6B4046FFF79DFF06442E604046F6
:101DB0007E68FFF797FF331A9C4203D801206C60BE
:101DC000BDE8F0816B603B68A61B0644AB60022057
:101DD000EE60F5E72046F3E738B50C460546FFF719
:101DE0009FFFA04210D305F10C00FFF77BFF0444D6
:101DF0006868BFF35B8FB4FBF0F100FB1144EC604B
:101E0000BFF35B8F012038BD0020FCE72DE9FF41C7
:101E10000F46694606466C46FFF7B6FF002504EB01
:101E2000C008444508D0626820687919FFF744FC6F
:101E3000636808341D44F4E729463046FFF7CCFFB9
:101E4000284604B0BDE8F081F8B505460C300F46D1
:101E5000FFF748FF05F1080604463046FFF742FF4A
:101E6000A042304688BF6C68FFF73CFF201A3860FC
:101E700020B130462C68FFF735FF2044F8BD000044
:101E8000F7B5174606460D46FFF732FFB84204463F
:101E900028BF3C460190DCB1304601A9FFF7D4FFD2
:101EA000019B33B93268C5E90233C5E9002401203A
:101EB0000CE09C4238BF019428600198844268601D
:101EC000F5D9241A02203368EC60AB6003B0F0BD92
:101ED0002046FBE72DE9FF410E466946FFF7D0FF9C
:101EE0006C46002504EBC007BC4209D0D4F804803E
:101EF0007019424654F8081BFFF7DEFB4544F3E730
:101F0000284604B0BDE8F08138B50546FFF7E2FF8A
:101F1000044601462846FFF71DFF204638BD000055
:101F2000302383F3118862B670470000002383F3E7
:101F3000118862B67047000010B4026854681A46EF
:101F4000234610BC1847000001207047002070474E
:101F50000020704770470000002070470E20704737
:101F600090F8C804C0F340007047000090F9C9041D
:101F700070470000F7B50C681E4614F00054BDF819
:101F800020706AD10B7B082B67D8FFF7C9FF456922
:101F9000AB685B010CD4AB681B0108D4AC6814F0CF
:101FA000805458D1FFF7C2FF204603B0F0BD012492
:101FB0000B6804F1180C002BBABFDB0043F00403DC
:101FC0005B054FEA0C1C45F80C300B684FEA041C0B
:101FD00013F0804F1CBF05EB0C0EDEF88031AC44D3
:101FE0001CBF43F00203CEF880310B7B05EB0415D8
:101FF000CCF884318B68C5F88C314B68C5F88831D2
:102000000D46DCF8803143F00103CCF8803100EB61
:102010004413C3F86824C3F86C6401F10C0C03F595
:102020008E6355F804EB654543F804EBF9D12D8830
:1020300024341D8000EB4414257907F0030325F0B8
:102040000B052B432371FFF771FF3346009700F018
:10205000BDFC0120A9E70224AAE74FF0FF30A4E766
:1020600038B50446D0F85C040D46FFF759FE1F282A
:102070000AD920222946D4F85C04FFF7C7FEA0F154
:1020800020035842584138BD0020FCE708B5FFF74F
:1020900047FFD0F85C04FFF719FEBDE80840FFF7E2
:1020A00045BF00000022026082814260826070476A
:1020B0000022002310B5C0E9002300230446038159
:1020C0000C30FFF7EFFF204610BD0000F0B590F890
:1020D000C8340D4613F0040FC3F3800108BF114646
:1020E00005F1240661F3820380F8C83400EB46133F
:1020F0001B790446D80789B02DD572B319072CD4A3
:1021000004EB45156846FFF7D3FF05F58E6303AA78
:1021100005F58F65174618685968083303C7AB4241
:102120003A46F7D11868694638609B882046BB80DC
:10213000DDE90E23CDE900230123ADF80830236843
:10214000DB6B984704EB461423791A075CBF43F016
:102150000803237101E0002AF4D109B0F0BD0000AA
:102160002DE9F047054688B068469A46884691466C
:10217000FFF7D6FEFFF79CFFD5F85C04FFF7B8FD2C
:102180001F282AD920226946D5F85C04FFF7BCFE37
:10219000202822D1444603AE05AB374603CF9F42E9
:1021A000206061603E4604F10804F6D1386841467B
:1021B0002060BB882846A380DDE90023C9E900230D
:1021C000BDF808304A46AAF80030FFF7AFFE534684
:1021D00008B0BDE8F04700F0E7BB0020FFF7A6FE1F
:1021E00008B0BDE8F087000000232DE9F047044661
:1021F000C0E90133224B0E4640F8183BFFF752FF6F
:1022000004F1480704F12800FFF752FF3D4604F5AA
:10221000896828462035FFF74BFF4545F9D14FF433
:102220008063C4F84874C4F84C34002701234FF08D
:1022300000084FF00009C4F85C54C4F85074C4F8A6
:10224000547484F8583484F8603404F5916504F5C6
:102250009D6A45E90889A5F11800FFF723FF20359D
:1022600045F8287C5545F4D184F8C96416B1054871
:1022700000F084FB044B20466361BDE8F08700BF9B
:1022800070470008484700080064004010B5044645
:10229000034B19784A1C1A70FFF7A6FF204610BDA1
:1022A000142300202DE9F04300294FD0284F294B5B
:1022B000B7FBF1F499428CBF0A231123B4FBF3FC62
:1022C000581E03FB1C43C5B22BB102280346F5D8A8
:1022D0000020BDE8F0830CF1FF36B6F5806FF7D231
:1022E0004FF47A74C5EBC50E0EF103034FEAE30910
:1022F00009FB0444C3F3C703E81AC0B209F101089B
:102300008044B4FBF8F4B4F5617FC2BF0EF1FF3333
:10231000C3F3C703E81A03F10104C8BFC0B2E4B2B3
:1023200004440CFB04F4B7FBF4F4A142D0D1013B0C
:10233000DBB20F2BCCD80138C0B20728C8D8002197
:102340001071168001209170D370C2E70846C0E773
:10235000005125023F420F0070B505460E464FF46E
:102360007A746B6901205B6803F00103B34204D007
:1023700001F080FC013CF4D1204670BD30B54269CB
:10238000936913F0700F16D000230B4C936103F187
:10239000240200EB421211794D0709D5890707D5B0
:1023A000416954F823508D60117941F00401117195
:1023B0000133032BEBD130BD5C47000873B51D46DC
:1023C000436916469A680446D20709D501219A68DE
:1023D0009960C2F340020021CDE90065FFF776FE67
:1023E00063699A68D1050BD54FF480719A682046CD
:1023F0009960C2F340220121CDE90065FFF766FE36
:1024000063699A68D2030BD54FF480319A682046ED
:102410009960C2F340420221CDE90065FFF756FE04
:10242000204602B0BDE87040FFF7A8BFF8B50446EB
:10243000466900296AD106F10C073868800768D020
:10244000386806EB01104FEA011CD0F8B011D0F843
:10245000B051490746BFED0845F000456D0DA56137
:10246000D0F8B011890744BF45F08045A561D0F888
:10247000B40106EB0C0100F00F0084F82400D1F841
:10248000B80104F124052077D1F8B801000A60777B
:10249000D1F8B801000CA077D1F8B801000EE077B0
:1024A000D1F8BC0184F82000D1F8BC01000A84F8FE
:1024B0002100D1F8BC01000C84F82200D1F8BC1135
:1024C00004F13400090E84F823103821396004F136
:1024D000180151F8046BA94240F8046BF9D109883E
:1024E0000180C4E90A2300232146238651F8283BB2
:1024F0002046DB6B984794F8C834204643F0040329
:1025000084F8C834BDE8F840FFF738BF06F110077B
:1025100093E7F8BD10B5044600F038FA02460B46C2
:1025200052EA030102D0013A63F10003044908684A
:1025300020B12146BDE81040FFF778BF10BD00BFB5
:1025400010230020F8B500211E46FFF7E9FC124FCA
:1025500000F58D6501F1240400EB4414237913F098
:10256000040F0FD1DB060DD5D5E900C39445B34167
:1025700008D2436957F821C0C3F808C0237943F053
:10258000040323710131032905F12005E2D1BDE8DF
:10259000F840FFF7CBBC00BF5C47000808B5FFF769
:1025A000BFFCFFF7EBFEBDE80840FFF7BFBC000033
:1025B000F8B54369044698680E4600F0E050B0F163
:1025C000E05F1DD0D8B1FFF7ABFC002504F58E67A6
:1025D00004EB451393F884341A0706D50135032D0F
:1025E00007F12007F4D1012007E05B07F6D4394654
:1025F000304600F025FA0028F0D1FFF797FCF8BD2F
:102600000120FCE708B5FFF78BFCD0F85C04FFF76E
:102610006FFBFFF78BFC43090CBF0120002008BDB6
:10262000F8B51D46002313700F4606461446FFF703
:10263000E9FF80F00100387025B129463046FFF7E8
:10264000B7FF2070F8BD0000F8B50C4615461E46D1
:10265000074600F09BF90B462178024609B9287815
:1026600050B13846FFF76EFFFFF798FF33462A4612
:102670002146FFF7D5FF0120F8BD000010B5FFF798
:102680004FFC174B0446DA6942F00072DA611A69AE
:1026900042F000721A611A6922F000721A61FFF7A3
:1026A00045FC90F8C834DB0718D4B9B103211320D6
:1026B000FFF736FC01F0ACF90321142001F0A8F972
:1026C0000321152001F0A4F994F8C83443F0010364
:1026D00084F8C834BDE81040FFF728BC10BD00BF27
:1026E000001002402DE9F04790F8C9340446012B50
:1026F0000F46154688B07DD87F4E56F823200AB97C
:1027000046F82300D6F80090E7602574B9F1000F71
:1027100062D094F8C934012B6ED04FF0000801212B
:102720002046FFF7ABFFFFF7FBFB6269012113684F
:10273000204623F0020313606269136843F001032B
:1027400013606369C3F81480FFF7F0FBFFF704FE22
:10275000002800F09280D4F85C04FFF7B7FAA14695
:1027600004F1600A202200216846FEF7B7FF02A8A4
:10277000FFF798FC6A46CDF8188009F58D630DF1D6
:10278000180C164603CE664518605960324603F1B0
:102790000803F6D1306809F1200918603279CA457A
:1027A0001A71DFD1002694F8C8346A466FF38203A9
:1027B00084F8C83439462046ADF80060ADF80260B0
:1027C0008DF80460FFF76EFD636948BB4FF400426B
:1027D0001A6008B0BDE8F0874FF49A6001F0DAFEA5
:1027E000804610B14946FFF7FFFCC6F80080B8F1FB
:1027F000000F8ED10020ECE7306803681B6B984710
:102800000146002889D13068FFF738FF30682A4632
:10281000036839465B68984700287FF47EAFE9E794
:102820006122022D0CBF4FF0004100211A609DF87B
:1028300002309DF803201B06120402F4702203F0FC
:1028400040731343BDF800202046C2F3090213432E
:102850009DF80420120502F4E002134362690B4361
:10286000D3611322636931465A616269136823F0A8
:1028700001031360FFF770FD08B96369A6E794F8D8
:10288000C93493BB6169D1F8002242F00102C1F85A
:1028900000226169D1F8002222F47C5222F00E025B
:1028A000C1F800226169D1F8002242F46062C1F8E7
:1028B000002241F6FF716269C2F814326269C2F8FF
:1028C00004326269C2F80C126269C2F8403262696D
:1028D000C2F8443201226369C3F81C226269D2F84B
:1028E000003223F00103C2F8003294F8C83443F0F8
:1028F000020384F8C8346CE71023002008B500F008
:1029000045F802460B4652EA030102D0013A63F150
:1029100000030449086808B1FFF750FDBDE808400E
:1029200001F054B81023002008B50020FFF7F2FD95
:10293000BDE8084001F04AB808B50120FFF7EAFDFC
:10294000BDE8084001F042B8EFF30983EFF30583D7
:10295000014B9B6BFEE700BF00ED00E008B5FFF701
:10296000F3FF0000EFF30983EFF30583014B5B6B8B
:10297000FEE700BF00ED00E0FEE700000FB408B581
:10298000029801F00DF9FEE701F0FABA01F0D2BAAF
:1029900013B56C4684E80600031D94E8030083E841
:1029A0000500012002B010BDF8B586680D4656B18D
:1029B0001B885B0707D4D0E900379B6B98472A46F2
:1029C000C1B23846B0470120F8BD0000F0B58668B6
:1029D00005460C4689B05EB1BDF838305B070AD4B5
:1029E000D0E900379B6B98472246C1B23846B047C2
:1029F000012009B0F0BD00220023CDE9002300230F
:102A00000A46ADF8083001F1080603AB1C46106811
:102A10005168083203C4B2422346F7D110682060DF
:102A20009288A280FFF7B2FF0423ADF808302B682C
:102A3000CDE90001DB6B694628469847D8E70000DE
:102A400030B503680968DD0FB5EBD17F23F0604432
:102A500021F060424FEAD1700BD0002BB8BFA40C1C
:102A60000029B8BF920C944202D034BF012000204C
:102A700030BD944205D1C1F38070C3F380738342AB
:102A8000F6D194422CBF00200120F1E72DE9F0415E
:102A9000456A15B94162BDE8F0814B68AC4623F048
:102AA0006047C3F38A4616EA230638BF3E464FEA1C
:102AB000D37EC3F380782B465A68BEEBD27F22F0D8
:102AC00060440AD0002A18DAA40CB44217D19D42FF
:102AD0000FD10D60DEE71346EEE7A74207D102F003
:102AE0008044C2F3807242450BD054B1EFE708D264
:102AF000EDE7CCF800100B60CDE7B44201D0B44252
:102B0000E5D81A689C46002AE5D11960C3E70000A1
:102B10002DE9F0474FF47F49089D01F007044FEA83
:102B2000D508224405F0070500EBD100944201D1FD
:102B3000BDE8F08704F0070705F0070A57453E4651
:102B400038BF5646111BC6F108068E4228BF0E46F6
:102B5000E108415C08EBD50E13F80EC0B94029FA24
:102B600006F721FA0AF1FFB28CEA010147FA0AF7E7
:102B700039408CEA010C03F80EC034443544D5E7E3
:102B8000082341F2210280EA012001B2400000291D
:102B900080B203F1FF33B8BF504013F0FF03F4D10C
:102BA0007047000038B50C468D18A54200D138BDDD
:102BB00014F8011BFFF7E4FFF7E700000346406845
:102BC00048B1026899895A605A89013292B2914299
:102BD0005A8138BF9A81704770B504460D4688B057
:102BE000202200216846FEF779FD20460495FFF774
:102BF000E5FF024658B16B46054608AE1C4603CCBD
:102C0000B44228606960234605F10805F6D11046F4
:102C100008B070BD082817D909280CD00A280CD094
:102C20000B280CD00C280CD00D280CD00E2814BF6B
:102C30004020302070470C2070471020704714202F
:102C4000704718207047202070470000082817D9C7
:102C50000C280CD910280CD914280CD918280CD9F8
:102C600020280CD930288CBF0F200E207047092057
:102C700070470A2070470B2070470C2070470D20CA
:102C8000704700002DE9F843078C0446072F1ED932
:102C9000D0E9029800254FF6FF73C5F12006A5F193
:102CA000200029FA05F108FA06F628FA00F0314367
:102CB0000143C9B21846FFF763FF0835402D0346AC
:102CC000EBD13A46E169BDE8F843FFF76BBF4FF639
:102CD000FF70BDE8F883000010B54B6823B9CA8ABD
:102CE00063F30902CA8210BD04691A681C6003619B
:102CF000C38A013BC3824A60EFE700002DE9F84F29
:102D00001D46CB8A0F46C3F3090105298146924629
:102D10000B4630D00020AAB207F11A049EB2042E4E
:102D20001FFA80F80FD8904503F1010306D3FB8A00
:102D30000A4462F309030120FB821AE01AF80060DA
:102D40000130E654EAE79045F1D21C23A1F1050BCE
:102D5000BBFBF3F203FB12BB7C681FFA8BF6002C63
:102D600045D14846FFF72AFF044638B978606FF02E
:102D70000200BDE8F88F4FF00008E6E70026066085
:102D800078604FF0000BADB2454510D90AEB08034F
:102D9000221D13F8011B08F101089155B1B21B293E
:102DA0001FFA88F82BD0454506F10106F1D8FB8AB9
:102DB000C3F30902154465F30903BCE71C4601325D
:102DC00092B22368002BF9D16B1F0B441C21B3FB7B
:102DD000F1F301339BB29A42D3D2BBF1000FD0D1B1
:102DE0004846FFF7EBFE20B9C4F800B0BFE7012268
:102DF000E7E7C0F800B05E4620600446C1E74545FD
:102E0000D5D94846FFF7DAFE08B92060AFE7C0F829
:102E100000B0002620600446B6E700002DE9F74F19
:102E20001C465B69074688460092002B00F097809D
:102E3000238C2BB1E269002A00F09180072B33D854
:102E400007F10C00FFF7BAFE054628B96FF002053E
:102E5000284603B0BDE8F08F14220021FEF73EFCA7
:102E6000228CE16905F10800FEF726FC208C48F071
:102E70000041013080B2FFF7E9FEFFF7CBFE0138D9
:102E800080B22084013028746369228C1B782A4424
:102E900003F01F0363F03F0313723846696029464D
:102EA000FFF7F4FD0125D3E74FF000094FF0800A4A
:102EB0004E464D4600F10C0301930198FFF77EFE4C
:102EC00083460028C2D014220021FEF707FC002E02
:102ED0003BD10222009BABF808300BF1080E1FFA21
:102EE00082FC0CF10100BCF1060F218C80B201D8EC
:102EF0008E422CD3FFF7AAFEFFF78CFE8E4208BF4E
:102F00004FF0400A62690138127880B202F01F0265
:102F100042EA49120BEB00014AEA020A013048F08A
:102F2000004281F808A08BF8100059463846CBF8CB
:102F30000420FFF7ABFD238C0135B3424FF0000AAC
:102F40002DB289F00109B8D182E70022C5E7E16915
:102F5000895D01360EF80210B6B20132BFE76FF09C
:102F6000010575E7F8B5044615460E4630220021E6
:102F70001F46FEF7B3FB069BB5F5001F6360079B7A
:102F800028BF4FF6FF72A3624FF0000338BF6A09F3
:102F9000A760E66197B204F110009A4206D80023B8
:102FA0000360A782E3822383E360F8BD06600133F8
:102FB00030462036F1E7000003781BB94BB2002BF6
:102FC000C8BF01707047000000787047F8B50C4624
:102FD000C969074611B9238C002B37D1257E1F2DD7
:102FE00034D8387828BB228C072A2CD8268A36F089
:102FF00003032BD14FF6FF70FFF7D4FD4FF6FF729E
:1030000020F001003602400446EA0565400C45EA1E
:103010004025234629463846FFF700FF002807DDF4
:10302000626913780133DBB21F2B88BF0023137052
:10303000F8BD218A2D0645EA012505432046FFF704
:1030400021FE0246E5E76FF00300F1E76FF00100B3
:10305000EEE7000070B504461D4616468AB02822E9
:1030600000216846FEF73AFBBDF838306946ADF8F6
:1030700010300F9B204605939DF84030CDE9026546
:103080008DF81830119B0793BDF84830ADF820300B
:10309000FFF79CFF0AB070BD2DE9F041D3690546EA
:1030A0000C4616460BB9138C5BBB377E1F2F28D8F6
:1030B00095F80080B8F1000F26D03046FFF7E2FD0A
:1030C0003378210241EAC33141EA0801338A41EAF7
:1030D000076141EA034102463346284641F0800138
:1030E000FFF79CFE00280ADD3378012B07D17269B7
:1030F00013780133DBB21F2B88BF00231370BDE8A8
:10310000F0816FF00100FAE76FF00300F7E70000CD
:10311000F0B504460D461E4617468BB02822002106
:103120006846FEF7DBFA9DF84C3029465A1E53429A
:1031300053418DF800309DF840306A46ADF81030AC
:10314000119B204605939DF84830CDE902768DF815
:103150001830149B0793BDF85430ADF82030FFF7BA
:103160009BFF0BB0F0BD0000406A00B10430704717
:10317000436A1A68426202691A600361C38A013BAA
:10318000C38270472DE9F041D0F8208014461D46D7
:1031900041460027174E09B9BDE8F081D1E9022365
:1031A000A21A65EB0303964277EB03031ED2036A70
:1031B0008B420DD1FFF790FD036A1B680362036920
:1031C0000B60C38A0161016A013B8846C382E2E762
:1031D000FFF782FD0B68C8F8003003690B60C38AF3
:1031E0000161013BC382D8F80010D4E78846096822
:1031F000D1E700BF80841E002DE9F04F8BB00D4653
:1032000014469B468046DDF85090002800F01A8155
:10321000B9F1000F00F01681531E3F2B00F212810E
:10322000012A03D1BBF1000F40F00C810023CDE94E
:103230000833B8F81430B5EBC30F4FEAC30703D314
:1032400000200BB0BDE8F08F2B199F42D8F80C304E
:1032500036BF7F1B2746FFB21BB9D8F81030002BB2
:103260007BD0272D4ED8C5F12806B7424FF000037A
:1032700034BF3E46F6B2009329463246D8F80800DD
:1032800008ABFFF745FCA7EB060A35445FFA8AFA5C
:103290002821B8F8143003F10053053BDB000493F8
:1032A000D8F80C300393039B13B1BAF1000F2CD163
:1032B000D8F8100040B1BAF1000F05D05246009680
:1032C00008AB691AFFF724FC38B2002FB8D06607A4
:1032D0000AD00AAB03EBD40111F8083C624202F0B9
:1032E0000702134101F8083C082C3DD9102C40F28C
:1032F000B680202C40F2B880BBF1000F00F09D801A
:10330000082335E0BA460026C2E7049BE02B28BF1D
:10331000E02306930B44AB42059315D95A1B924503
:1033200038BF5246039828BFD2B20096691A08AB3C
:1033300004300792FFF7ECFB079A1644AAEB020A47
:103340001544F6B25FFA8AFA049B069A05999B1A0D
:103350000493039B1B680393A5E700933A46294611
:10336000D8F8080008ABADE7BBF1000F13D001237C
:10337000B4EBC30F6CD0082C12D89DF82030621E1D
:1033800023FA02F2D50706D54FF0FF3202FA04F411
:1033900023438DF820309DF8203089F8003050E725
:1033A000102C12D8BDF82030621E23FA02F2D10789
:1033B00006D54FF0FF3202FA04F42343ADF8203073
:1033C000BDF82030A9F800303BE7202C0FD8089931
:1033D000631E21FA03F3DA0705D54FF0FF3202FA34
:1033E00004F40C430894089BC9F8003029E7402CEA
:1033F0002BD0DDE90865611EC4F12102A4F121038F
:1034000026FA01F105FA02F225FA03F311431943F2
:10341000CB0712D50122A4F12003C4F1200102FA46
:1034200003F322FA01F1A240524243EA010363EBA3
:10343000430332432B43CDE90823DDE90823C9E9DF
:103440000023FEE66FF00100FBE66FF00800F8E6EF
:10345000082CA0D9102CB3D9202CEED8C3E7BBF18F
:10346000000FADD0022383E7BBF1000FBBD00423D4
:103470007EE70000012A30B5144638BF012200253E
:10348000402A28BF402285B0012CCDE9025517D82B
:103490001B788DF8083053070AD004AB03EBD20534
:1034A00015F8083C544204F00704A34005F8083C12
:1034B0000346009102A80021FFF72AFB05B030BDAA
:1034C000082CE5D9102C03D81B88ADF80830E2E7AA
:1034D000202C02D81B680293DDE7D3E90045CDE933
:1034E0000245D8E710B5CB681BB98B600B618B82A6
:1034F00010BD04691A681C600361C38A013BC38262
:10350000CA60F0E703064CBFC0F3C030022070472A
:1035100008B50246FFF7F6FF022806D15306C2F3AC
:103520000F2001D100F0030008BDC2F30740FBE704
:103530002DE9F04F93B0CDE903230A680446104605
:10354000FFF7E0FF02280CBF0026C2F30626002A80
:103550000D46824680F2F98112F0C04940F0F581B3
:10356000097B002900F0F181022803D02378B342BF
:1035700040F0EE81C2F304631046069302F07F032D
:103580000593FFF7C5FF059B00224FEA8348002300
:1035900048EA0A48294448EA4668CE78CDE9082333
:1035A000F309834648EA0008029367D0059B024668
:1035B000009320465346676808A9B847002800F0E2
:1035C000CA81276A4FB9414604F10C00FFF704FB9A
:1035D000074690B96FF0020054E03B6998450DD062
:1035E0003F68002FF9D1414604F10C00FFF7F4FACF
:1035F00007460028EED0236A3B60276297F817C081
:1036000006F01F08CCF3840CACEB08001FFA80FE18
:103610000028B8BF0EF12000A8EB0C031FFA83FEB0
:10362000B8BF00B2002B0793BEBF0EF120031BB240
:103630000793D7E9022152EA010338D04FF0000C7A
:10364000039BDFF8F8E19A1A049B63EB01019645AE
:103650007CEB01032BD36B7B97F81AE0734519D1F0
:10366000029B002B78D0012821DC7868F8B9DFF8BC
:10367000D0C1944570EB010316D337E0276A27B910
:103680006FF00C0013B0BDE8F08F3B699845B5D0E2
:103690003F68F4E76A4890427CEB010301D30020C5
:1036A000F0E7029B002BFAD0079B0F2B17DCFA7D6B
:1036B000B30002F0030203F07C031343FB753946A9
:1036C0002046FFF709FB6B7BBB76029B3BB9FB7D7A
:1036D000C3F38402013262F38603FB75D0E76A7B91
:1036E000BB7E9A42DBD1029B002B35D0B309022B63
:1036F00032D0039B1422BB60049B0021FB600DA809
:10370000FDF7ECFF039B20460A93049BADF83EB007
:103710000B932B1D0C932B7B8DF840A0013BDBB250
:10372000ADF83C30069B8DF841808DF84230059B0A
:103730000AA98DF8433094F82C3083F001038DF8FA
:103740004430A3689847FB7DC3F38403013303F03F
:103750001F039B02FB82A2E7FB7DC6F34012B2EB84
:10376000D31F40F0FB80C3F38403434540F0F9804E
:10377000029A2B7BB609002A4DD0F20762D4032BA4
:1037800040F2F280039BAE1DBB60049B3246FB609F
:103790002B7B3946033BDBB204F10C00FFF7AEFA9A
:1037A00000280CDA39462046FFF796FAFB7DC3F372
:1037B0008403013303F01F039B02FB820AE7AB88FB
:1037C000DDE908843B834FF6FF73C9F12000A9F1BE
:1037D000200228FA09F104FA00F0014324FA02F267
:1037E00011431846C9B2FFF7CBF909F10809B9F13D
:1037F000400F0346E9D13146B8822A7B033AD2B260
:10380000FFF7D0F9FB7DB882DA43C2F3C01262F34E
:10381000C713FB7543E7AEB92E1D013B324639464F
:10382000DBB204F10C00FFF769FA0028BADB2A7B4F
:103830003146013AB88AD2B2E2E700BF80841E0066
:1038400040420F00F98A013BC1F309010429DAB2B1
:103850005DD80023281D07F11B069A4208D910F8ED
:1038600001CB013306F801C001310529DBB2F4D1E7
:10387000934228BF0023039938BF04330A91049967
:1038800038BFDBB20B9107F11B010C91796838BF8F
:103890005B190D910E93FB8AADF83EB0C3F309039B
:1038A0001A44069BADF83C208DF84230059B8DF8FC
:1038B00040A08DF8433094F82C308DF8418083F08F
:1038C00001038DF8443000237B602A7BB88A013ADB
:1038D000291DFFF767F93B8BB882834203D120464D
:1038E000A3680AA9984720460AA9FFF7FBFDFB7DBC
:1038F000BA8AC3F38403013303F01F039B02FB82E4
:103900003B8B9A420CBF00206FF01000BAE67B6838
:10391000002BADD0052001E033461C301E68002E80
:10392000FAD1091A081D2E1D184401EB090CBCF12F
:103930001B0F5FFA89F39BD89A4299D916F8013B7D
:1039400009F1010900F8013BEFE76FF0090099E682
:103950006FF00A0096E66FF00B0093E66FF00D0033
:1039600090E66FF00E008DE66FF00F008AE600BF64
:10397000EFF30983203383F30988002383F311884D
:1039800070470000302080F3118862B60C4B0D4A5E
:10399000D96821F4E0610904090C0A43DA60D3F81C
:1039A000FC20094942F08072C3F8FC200A6842F00A
:1039B00001020A602022DA7783F82200704700BFF4
:1039C00000ED00E00003FA05001000E0302310B520
:1039D00083F311880B4B5B6813F400630FD0EFF394
:1039E00009844FF08073203CE36184F3098800F080
:1039F00095F810B1044BA36110BD044BFBE783F3B2
:103A00001188F9E700ED00E03F09000842090008CD
:103A10000122090100F1604303F56143C9B283F853
:103A2000001300F01F039A4043099B0003F1604319
:103A300003F56143C3F880211A607047090100F162
:103A40006040C9B200F56D4001767047002382687E
:103A5000037503691B6899689142FBD25A68036039
:103A600042601060586070470023826803750369E4
:103A70001B6899689142FBD85A68036042601060E5
:103A80005860704708B50846302383F311880B7DD2
:103A9000032B05D0042B0DD02BB983F3118808BD5F
:103AA00000228B691A604FF0FF338361FFF7CEFF6E
:103AB0000023F2E7D1E9003213605A60F3E7000017
:103AC000FFF7C4BF054BD9680875186802685360D2
:103AD0001A6001220275D860FCF720BF2023002065
:103AE00030B50C4B0446DD684B1C87B00FD02B461D
:103AF0006846094A00F0E2F82046FFF7E3FF009B22
:103B000013B1684600F0E2F8A86907B030BDFFF7CE
:103B1000D9FFF9E720230020853A0008044B1A68F2
:103B2000DB6890689B68984294BF00200120704732
:103B300020230020084B10B51C68D8682268536009
:103B40001A6001222275DC60FFF78EFF01462046D5
:103B5000BDE81040FCF7E2BE20230020044B1A68A9
:103B6000DB6892689B689A4201D9FFF7E3BF704710
:103B70002023002038B501230025064C06490748BC
:103B80002370656000F0D8FA0223237085F3118852
:103B900038BD00BF78240020B4470008202300204F
:103BA00008B572B6044B186500F0B2F900F056FA89
:103BB0000322024B1A70FEE7202300207824002005
:103BC00000F096B8EFF3118020B9EFF305833022AF
:103BD00082F311887047000010B530B9EFF3058407
:103BE000C4F3080414B180F3118810BDFFF7B6FFC9
:103BF00084F31188F9E700008B60022308618B824F
:103C0000084670478368A3F1440243F8142C026904
:103C100043F8442C426943F8402C094A43F8242CC9
:103C2000C268A3F1200043F8182C022203F80C2CE0
:103C3000002203F80B2C034A43F8102C704700BFF6
:103C40002D0900082023002008B5FFF7DBFFBDE8A1
:103C50000840FFF735BF0000024BDB6898610F207A
:103C6000FFF730BF20230020302383F31188FFF7B4
:103C7000F3BF000008B50146302383F31188082004
:103C8000FFF72EFF002383F3118808BD10B50A4CFF
:103C900023699A6891420CD85A6881600360426037
:103CA00010609A685860511A99604FF0FF33A36111
:103CB00010BD1B68891AECE720230020C0E903230C
:103CC000002310B410BC4361FFF7E0BF03688168B4
:103CD0009A680A449A60426813605A6000234FF061
:103CE000FF320360014B9A61704700BF2023002020
:103CF00070B5124D2A46EB690133EB6152F8103F63
:103D0000934206D030269A68013A9A602C69A368DB
:103D100003B170BDD4E900210A605160236083F3D0
:103D200011882046D4E90331984786F311886169E8
:103D30000029EBD02046FFF7A9FFE7E7202300206A
:103D400000207047FEE70000704700004FF0FF3092
:103D500070470000BFF34F8F024AD368DB07FCD4E3
:103D6000704700BF0020024008B5074B1B7853B9CD
:103D7000FFF7F0FF054B1A69120641BF044A5A606B
:103D800002F188325A6008BD9024002000200240D1
:103D90002301674508B5054B1B7833B9FFF7DAFFF8
:103DA000034A136943F08003136108BD9024002087
:103DB000002002407F289ABF00F58030C00200201A
:103DC000704700004FF4006070470000802070478B
:103DD0007F2808B50BD8FFF7EDFF00F500630268F8
:103DE000013204D104308342F9D1012008BD002002
:103DF000FCE700007F2810B504461CD8FFF7AAFF97
:103E0000FFF7B2FFF3220D4B4FF40061DA6002229C
:103E10001A61FFF7CFFF58611A6942F040021A6138
:103E2000FFF798FF00F016F9FFF7B4FF2046BDE852
:103E30001040FFF7CDBF002010BD00BF00200240A2
:103E40002DE9F843054612F00100144606D040F271
:103E5000F32200201E4B1A60BDE8F8831D4BAA1800
:103E60009A4204D94FF43E72194B1A60F4E7FFF7F7
:103E70007BFF4FF00109FFF76DFFDFF85C806D1AE3
:103E8000012C0F4605EB010603D8FFF783FF012045
:103E9000E2E73B88C8F8109033800020FFF75AFF14
:103EA000C8F81000338831F8022B9BB29A420CD02C
:103EB00040F20F32064B1A60084B1E60084B1C6024
:103EC000084B1F60FFF766FFC6E7023CD8E700BF5C
:103ED0008C240020000004080020024080240020E0
:103EE0008824002084240020084908B50B7828B1D4
:103EF0001BB9FFF739FF01230B7008BD002BFCD065
:103F0000BDE808400870FFF745BF00BF90240020BF
:103F10004FF480314FF0005000F09EB80846114633
:103F200000F05ABB012000F057BB0000084600F02B
:103F300071BB000070B5FFF745FE4FF47A710D4B71
:103F40000D4EDB69326801FB03F3934237BF0B4A26
:103F50000A495168156836BF4C1CD1E900545460B9
:103F60005D1944F100043360FFF736FE2846214610
:103F700070BD00BF2023002094240020982400203E
:103F800070B5FFF71FFE4FF47A710F4B0F4EDB69D0
:103F9000326801FB03F3934237BF0D4A0C49516865
:103FA00015683ABF4C1C5460D1E900545D1944F1C6
:103FB00000043360FFF710FE4FF47A7200232846A6
:103FC0002146FCF7B7FA70BD20230020942400207E
:103FD0009824002010B5094C013AD2B2FF2A00D132
:103FE00010BD500854F82030013054F820009BB226
:103FF00043EA004341F8043BEEE700BF046C004095
:1040000010B50748013AD2B2FF2A00D110BD0C8882
:10401000530840F823404C88013340F82340F1E72F
:10402000046C004007B50122002001A9FFF7D2FF70
:10403000019803B05DF804FB13B50446FFF7F2FFE7
:10404000A04205D00122002001A90194FFF7D8FF6A
:1040500002B010BD704700007047000070470000BC
:1040600045F25552064B1A6002225A6040F6FF7222
:104070009A604CF6CC421A600122024B1A707047CB
:1040800000300040A4240020034B1B781BB14AF6EB
:10409000AA22024B1A607047A4240020003000407E
:1040A000044B1A682AB902F1804202F50432526ABE
:1040B0001A607047A02400204FF08072014B5A62B2
:1040C000704700BF0010024008B5FFF7E9FF024B40
:1040D0001868C0F3407008BDA024002008B5FFF7A1
:1040E000DFFF024B1868C0F3007008BDA024002059
:1040F00070470000FEE700000A4B0B480B4A904255
:104100000BD30B4BC11EDA1C121A22F003028B4296
:1041100038BF00220021FDF7E1BA53F8041B40F834
:10412000041BECE7904800083025002030250020D3
:1041300030250020FEE7000070B5002504461A4B2C
:1041400086B05860856201630E46FFF71BFC04F1E0
:104150001003C4E904334FF0FF33A361134BE5614F
:10416000D9692B460A462046C4E9082304F13401E4
:104170008023C4E900440E4AA560E5622565FFF787
:104180003BFD01230B4AE0600375009272686846AC
:104190000192B268CDE90223074BCDE90435FFF760
:1041A00053FD06B070BD00BF7824002020230020FE
:1041B000C0470008C54700083541000800F030B886
:1041C00008B500F06DF9FFF7D5FCBDE80840FFF732
:1041D00067BF0000704700004FF0FF310E4B1A69B7
:1041E00019611A6900221A611869D868D960D968FA
:1041F000DA60DA68DA6942F08052DA61DA69DA693B
:1042000042F00062DA61054ADB69136843F48073A7
:10421000136000F025B900BF00100240007000409C
:104220001E4B1A6842F001021A601A689007FCD50A
:104230005A6822F003025A605A6812F00C02FBD14D
:10424000196801F0F90119605A601A6842F4803265
:104250001A601A689103FCD54EF63162DA625A6828
:1042600042F4E8125A601A6842F080721A601A68C2
:104270009201FCD50A4A0B495A6012220A600A6868
:1042800002F00702022AFAD15A6842F002025A608A
:104290005A6802F00C02082AFAD170470010024056
:1042A00000641D0000200240084A08B551691368E7
:1042B0000B4003F00103536123B1054A13680BB1AE
:1042C00050689847BDE80840FFF780BB00040140F4
:1042D000A8240020084A08B5516913680B4003F070
:1042E0000203536123B1054A93680BB1D068984724
:1042F000BDE80840FFF76ABB00040140A824002085
:10430000084A08B5516913680B4003F00403536170
:1043100023B1054A13690BB150699847BDE80840BD
:10432000FFF754BB00040140A8240020084A08B548
:10433000516913680B4003F00803536123B1054A28
:1043400093690BB1D0699847BDE80840FFF73EBBC1
:1043500000040140A8240020084A08B551691368E8
:104360000B4003F01003536123B1054A136A0BB1EC
:10437000506A9847BDE80840FFF728BB0004014099
:10438000A8240020174B10B55A691C68144004F487
:1043900078725A61A30604D5134A936A0BB1D06AA6
:1043A0009847600604D5104A136B0BB1506B9847C1
:1043B000210604D50C4A936B0BB1D06B9847E205EC
:1043C00004D5094A136C0BB1506C9847A30504D56A
:1043D000054A936C0BB1D06C9847BDE81040FFF7CD
:1043E000F5BA00BF00040140A82400201A4B10B504
:1043F0005A691C68144004F47C425A61620504D571
:10440000164A136D0BB1506D9847230504D5134A16
:10441000936D0BB1D06D9847E00404D50F4A136E2D
:104420000BB1506E9847A10404D50C4A936E0BB1A2
:10443000D06E9847620404D5084A136F0BB1506FD1
:104440009847230404D5054A936F0BB1D06F984762
:10445000BDE81040FFF7BABA00040140A8240020CC
:10446000062108B50846FFF7D3FA06210720FFF713
:10447000CFFA06210820FFF7CBFA06210920FFF723
:10448000C7FA06210A20FFF7C3FA06211720FFF713
:10449000BFFABDE8084006212820FFF7B9BA00009E
:1044A00008B5FFF799FE044800F00AF8FFF792FEFE
:1044B000BDE8084000F002B8CC47000800F042B860
:1044C000002319461C4A0133102BC2E9001102F1E6
:1044D0000802F8D1194B9A6942F07D029A619B69F2
:1044E0000268174BDA6082685A6042681A60C268D4
:1044F00003F58063DA6042695A6002691A60826972
:10450000C3F80C24026AC3F80424C269C3F8002467
:10451000426AC3F80C28C26AC3F80428826AC3F846
:104520000028026BC3F80C2C826BC3F8042C426B7E
:10453000C3F8002C704700BFA824002000100240E0
:10454000000801404FF0E023044A08215A6100228C
:104550009A6107220B201A61FFF770BA3F19010018
:1045600008B5302383F31188FFF72AFB002383F378
:10457000118808BD08B5FFF7F3FFBDE80840FFF755
:1045800025BA00000B460146184600F02DB8000081
:1045900000F040B8012838BF012010B5044620467D
:1045A00000F030F830B900F007F808B900F00CF866
:1045B0008047F4E710BD0000024B1868BFF35B8F23
:1045C000704700BF28250020062008B500F082F8BB
:1045D0000120FFF7B7FB0000024B0A4601461868AE
:1045E000FFF79CBC1C08002010B504460448134685
:1045F00020B10A4602202146AFF3008010BD00BF63
:1046000000000000024B01461868FFF78BBC00BF9A
:104610001C080020024B01461868FFF787BC00BF4A
:104620001C08002010B501390244904201D100203D
:1046300005E0037811F8014FA34201D0181B10BD0B
:104640000130F2E72DE9F0419BB10446C91A177811
:10465000014403F1FF3C8C42204601D9002008E0D0
:1046600005780134BD42F6D10CEB0405D618A542FD
:1046700001D1BDE8F08115F8018D16F801EDF04586
:10468000F5D0E8E71F2938B504460D4604D91623AE
:1046900003604FF0FF3038BD426C12B152F8213048
:1046A0004BB9204600F030F82A4601462046BDE8C6
:1046B000384000F017B8012B0AD0591C03D116233B
:1046C00003600120E7E70024284642F82540984788
:1046D0000020E0E7024B01461868FFF7D3BF00BF98
:1046E0001C08002038B50023064D04460846114634
:1046F0002B60FFF72BFB431C02D12B6803B1236017
:1047000038BD00BF2C250020FFF71ABB034611F867
:10471000012B03F8012B002AF9D170476F72672E25
:104720006172647570696C6F742E5A756261784736
:104730004E53530040A2E4F1646891060041A3E5A2
:10474000F2656992070000004261642043414E49CE
:104750006661636520696E6465782E0080000000E4
:104760000080000000008000000000000000000049
:10477000391F0008E526000849260008491F0008DF
:10478000751F0008612100084D1F00085D1F00080B
:10479000511F0008591F0008551F00088D200008F0
:1047A000611F0008912900086D1F000861200008A2
:1047B00063300000B04700087823002078240020F0
:1047C0006D61696E0069646C650000000C88000012
:1047D000447B444444544424800E00004414111487
:1047E000947B444400000000444444444444444412
:1047F0000400000044424444444444440000000097
:1048000044444444444444445CBDFF7F01000000F0
:10481000ED0300000000000000680300000000003D
:1048200040420F00FE2A0100D204000020080020B0
:104830000000000000000000000000000000000078
:104840000000000000000000000000000000000068
:104850000000000000000000000000000000000058
:104860000000000000000000000000000000000048
:104870000000000000000000000000000000000038
:104880000000000000000000000000000000000028
:00000001FF
